:100000008B01831684308100143085000130860016
:1000100083120230850086010830A500A601030185
:10002000FF3E031D1028051A0028A60F1028A50B57
:1000300010280C3084008001840A041F1B28051D31
:10004000272885100000000005192728B82B8316E3
:100050001030850083125B2301309F0007309E0023
:100060009F178C1581010B11051A2D2B0B1941209F
:100070000C1D34288C300106031D34288510051111
:10008000342864308100900A101DB028810390014B
:10009000061C04210C1F5B288B1C5B288316011394
:1000A00083128B100C131308033C03185B281308EE
:1000B000313C03181A29910A32301106031D832896
:1000C0009101940A3C301406031D83289401960A7A
:1000D00017081606031D802896010310180CF62039
:1000E000DD201A08AA00AB01E92003187D280310BF
:1000F000180CF620DD20FF2080281A088F008E01C2
:100100009D08031D9D038C19CE281D0A03199D28E7
:100110008C121A080F0203188C169D08031DA328C1
:1001200085110C150C108C100C160F0803100E18EE
:10013000031431238C1A9E17B028D62294010C1573
:100140000C108C10B02885150C110C120C108C1092
:100150001D0831231D08053C031CB0280C148C1409
:1001600085100511051001308605101CC2281F08D6
:10017000D82386049F1B05141930110203188C1C08
:100180000515CC281E08D82386049E1B051419309B
:10019000110203180C1C85140B1108000D08033CF8
:1001A000031CB028920AFA301206031DB0289201EF
:1001B0008C118D010C108C1083280130A905AB0522
:1001C0002B08A907A918A80AA9102A08A80728080F
:1001D00008000130A905AB05A9142B08A902A91C28
:1001E000AA0AA9102A08A80228080800AA00AB0138
:1001F00003182B140F08A8000E08A90008002808EF
:100200008F0029088E0008008B1C0C29930183168F
:10021000011783128B100C17930A3230130603193F
:100220003A29963013060319AA2AFF301306031938
:100230009303080001308A0016300D0203180800ED
:100240000D08031D9101820758298F298F298F29B5
:10025000BC2ABC2ABC2ABC2ABC2ABC2ABC2ABC2A6E
:10026000B72A08009629A729B029BF29CB298F29A9
:100270008F298F2901308A0016300D0203180800DB
:100280000D088207942AD429E029EB29F529FF29B2
:10029000032A162A342A432A5B2A6C2AA02AA02A77
:1002A0000F2A1E2A3B2A4A2A622A752A7C2A832A76
:1002B0001B081D020318080063301D023C30031C9C
:1002C0001C08A100210A1D070318A10221081D070F
:1002D0001B02031CA1070310210CF620E920031CBC
:1002E0007C290310210CF620E920FF209D0803192A
:1002F000940121089D0708009D0803190800A10129
:100300008F080319A10A0E1CA10AA11808000310E6
:100310000F0D9D070E189D0A8F018E010800920196
:100320009E0A0A301E0603199E0108001E30A3070C
:100330000318A42123081A02031CA4212308031074
:100340002418031431230800A401A30108001E305F
:10035000A3073C300318A30023080310312308002F
:100360000530A30723083C3C0530031CA3002308E9
:100370001B020530031CA30023083123080078303A
:1003800023023C30031C1E30A3071E300318A300B9
:10039000230831230800A30A23080F3C0130031C63
:1003A000A30023083123080092018C173D30B123AC
:1003B000A5001E06031D8C138D0A9F0A9E010800CE
:1003C00092013E30B123A6001E06031D8C138D0A38
:1003D0009F0A9E01080092013F30B123A7001E062C
:1003E000031D8C138C1FA02AB72A0D308D000B30F3
:1003F0009F0011309E000C108C108515A72AFF302D
:100400009D009C23A02A0E308D000E08A4000F082A
:10041000A3000C160310241803143123080023082A
:100420008F0024088E0006308D00BD2A0F308D000D
:100430001A08A3000C1603103123080023089A00A1
:1004400088000130CA231A08A800A9010F08AA00D1
:100450000E08AB00E920031C302207308D00BD2AB6
:100460001A088F008E01080010308D001C08A300B0
:100470000C123123080023089C0088000330CA2393
:1004800008308D00BD2A11308D001B08A3000C120E
:100490003123080023089B0088000230CA231C086F
:1004A00023022308031C9C001C0888000330CA2375
:1004B00009308D00BD2A12308D001908A3000C12DE
:1004C000312308002308990088000301CA23FE2273
:1004D00096010A308D00BD2A13308D0001309F0037
:1004E0009F178C1025089E0008001E08A5008D0A85
:1004F0009F0A26089E0008001E08A6008D0A9F0A73
:1005000027089E0008001E08A700250888003D3027
:10051000CA23260888003E30CA23270888003F30B7
:10052000CA230B308D00BD2A1D0A031908009D083F
:100530000319080003101D0CF620DD20FF209D018B
:100540008D01A501A601A7018C110C108C10FE30A5
:10055000930008008D08031DA02A01308D009F0024
:100560009F178C150C140C119E01920108009D011F
:100570009C2304308D00BD2A8D0A0C148C1402308B
:100580008A0004300D020F398207D12AD62ADB2ACD
:10059000E02AE52AEA2AEF2AF42AF92A08000800C4
:1005A00008000B309F0011309E0008000B309F00A8
:1005B0000F309E0008000E309F0012309E00080091
:1005C0000E309F000F309E00080013309F000C304B
:1005D0009E00080013309F000F309E00080014306A
:1005E0009F0015309E0008000D309F0010309E00C7
:1005F00008000B309F0012309E0008000323970074
:1006000018239800080003308A000F30190582076C
:10061000FF3418340C3408340634183404341834D5
:10062000033408340C341834023418340C340834CD
:1006300003308A000F301905820700340134013479
:1006400001340134053401340734013403340534F2
:100650000B3401340D3407340534850186019C23A5
:100660000028A201031822149F019E0064300C1A76
:1006700032301E02031C482B3C300C1A1E301E0266
:10068000031C452B9E009F0A3C2B0A309E00592BD1
:100690000C1E4E2B03109E0D22181E140A301E0233
:1006A000031C552B9E009F0A4E2B0B309F080319ED
:1006B0009F00030108000301C42399000130C423F3
:1006C0009A000230C4239B000330C4239C000430F2
:1006D000C4238E000530C4238F000630C423960047
:1006E0000730C4239D000830C423940019080F3C30
:1006F0000330031C9900FE221B08F03C7830031CD9
:100700009B001A08F03C3C30031C9A001C083C3C3F
:100710001E30031C9C0016081702031C96011408C7
:100720003B3C031C94010E08013C031C8E010F0886
:100730001A0203180800302A0E0888000430CA2361
:100740000F0888000530CA23160888000630CA231F
:100750001D0888000730CA23140888000830CA23FF
:100760000800C423A100093C031CA10121080800C2
:1007700088013D30CA2388013E30CA2388013F30BA
:10078000CA2305148514C32B890083160814831209
:1007900008080800890083160815081255308900DA
:1007A000AA3089008814081ED32B08118312080070
:1007B000A0001F30A00503308A0016302002031865
:1007C0000034200882077E340C34B6349E34CC3496
:1007D000DA34FA340E34FE34DE34E8340034EE34E5
:1007E0007234EC347034B834E634F2347C34BC34D3
:0207F000F034E3
:02400E000100AF
:1042000003003C0078001E0000003C00000000009D
:024210000000AC
:06427A000000000000003E
:00000001FF
